:020000040000FA
:04000000D1303A2899
:08000800A000030EA100831209
:1000100005191028831601178312B23081002B288E
:1000200083160113831203140B190310A80DA90DD5
:10003000AA0DAB0DAC0DAC16FF302C02031D2B2806
:10004000FA302B02031D2B2831152A08AF0029088E
:10005000AE002808AD008B100B11210E8300A00EFE
:04006000200E090065
:0C007400203084008001840A80300402E7
:10008000031C3C281230B000F82183160C30850583
:1000900087018312850187010730990000309A009B
:1000A000103083168E008312603083168F00831207
:1000B0000030831691009F008312C83083168100A0
:1000C000831231309000003083168C008312103080
:1000D0008B00831600309B001C141A088312BC008E
:1000E000831610309B001C141A088312BD0083165F
:1000F00030309B001C141A088312DE005D2381013E
:100100008E018F010B118B100B108C018B17962019
:1001100031199920B30B9428031085190314B90DD4
:10012000F030390203195421A023872864003210CB
:10013000080031110130B7008B13203037078316C8
:100140009B001C141A088312A40010303707831672
:100150009B001C141A088312A300A6000230A606F6
:100160000030370783169B001C141A088312A20064
:10017000A7000130A7068B17321CC42822090339B7
:10018000A200A309A409A50924082F02031D4E29D2
:1001900023082E02031D4E2922082D02031D4E297D
:1001A00001303702031DD9283D18D9283D143E14CB
:1001B000052202303702031DE228BD18E228BD14D3
:1001C0003E14172203303702031DEB283D19EB289C
:1001D0003D153E14292204303702031DF428BD19B1
:1001E000F428BD153E143B2205303702031DFD28BF
:1001F0003D1AFD283D163E144D2206303702031DE0
:100200000629BD1A0629BD163E145E2207303702A4
:10021000031D0F293D1B0F293D173E146F22083087
:100220003702031D1829BD1B1829BD173E14802253
:1002300009303702031D21295E1821295E143E145E
:1002400091220A303702031D2A29DE182A29DE14DA
:100250003E14AA220B303702031D33295E193329BD
:100260005E153E14C3220C303702031D3C29DE19F3
:100270003C29DE153E14D8220D303702031D4529D6
:100280005E1A45295E163E14ED220E303702031D1C
:100290004E29DE1A4E29DE163E140223B70A0F300D
:1002A0003702031808009C280130B600B300B400E0
:1002B000B500B70085018701B1139620B30BA429BF
:1002C000031085190314B90DF03039020319CB2935
:1002D000B40BA42901303702031917230230370267
:1002E00003191C230330370203192123043037027A
:1002F000031926230530370203192B230630370252
:100300000319302307303702031935230830370229
:1003100003193A230930370203193F230A30370201
:10032000031944230B303702031949230C303702D9
:1003300003194E230D303702031953230E303702B1
:10034000031958239630B400311D5D293111321C38
:10035000AE292D090339AD00AE09AF092F1C5D2967
:100360008E018F010C1C5D290C102E1E5D298B1334
:1003700020303707BB002F08BA00E32110303707C1
:10038000BB002E08BA00E32100303707BB002D0860
:10039000BA00E3218B1785018701B70AB6010F3038
:1003A0003702031C5D295D2308003E1C08003E1037
:1003B0001030BB003D08BA00E3213030BB005E08BE
:1003C000BA00E32108008B133A0883161C159A0023
:1003D00083123B0883169B0055309D00AA309D0078
:1003E0009C1464009C18F1291C1183128B170800BF
:1003F000FF30C800CA15CB15CC15CD15CE15CF15BD
:10040000D015D115D215D31508000130BD05003027
:10041000DE054030C405C0000030C200C6004030D8
:10042000C505C1000030C300C7005F1008000230DE
:10043000BD050030DE050830C405C0000030C20034
:10044000C6004030C505C1000030C300C7005F10C2
:1004500008000430BD050030DE050830C405C000CA
:100460000030C200C6004030C505C1004030C300A6
:10047000C7005F1008000830BD050030DE05883079
:10048000C405C0000030C200C6000030C505C10070
:100490000030C300C7005F1008001030BD050030F9
:1004A000DE058830C405C0008030C200C6000030C0
:1004B000C505C1000030C300C70008002030BD05DD
:1004C0000030DE051030C405C0000030C200C60098
:1004D0000030C505C1000030C300C700080040302F
:1004E000BD050030DE052030C405C0000030C2006C
:1004F000C6000030C505C1000030C300C7000800B9
:100500008030BD050030DE052030C405C00020303D
:10051000C200C6000030C505C1000030C300C700DE
:1005200008000030BD05C130DE0508304418013A2E
:10053000C418023AC405C00000304618013AC61873
:10054000023AC200C6008030C505C1000030C300B9
:10055000C70008000030BD05C230DE050830441871
:10056000013AC418023AC405C00000304618013AE6
:10057000C618023AC200C6008030C505C1008030EE
:10058000C300C70008000030BD05C430DE050A30D6
:10059000C405C0000030C200C6000030C51B803A50
:1005A000C505C1000030C71B803AC300C700080062
:1005B0000030BD05C830DE050A30C405C000023079
:1005C000C200C6000030C51B803AC505C10000301E
:1005D000C71B803AC300C70008000030BD05D030FB
:1005E000DE050930C405C0000030C200C60000307E
:1005F000C51B803AC505C1000030C71B803AC30047
:10060000C70008000030BD05E030DE050930C40534
:10061000C0000130C200C6000030C51B803AC505CD
:10062000C1000030C71B803AC300C700080000307B
:1006300085061130870608000230850610308706CF
:100640000800023085061030870608000230850653
:100650002030870608000230850620308706080013
:100660000030850602308706080000308506043019
:10067000870608000030850604308706080002302F
:100680008506083087060800023085060830870690
:1006900008002230850600308706080022308506D3
:1006A00000308706080012308506003087060800F3
:1006B000123085060030870608003D180522BD1857
:1006C00017223D192922BD193B223D1A4D22BD1A80
:1006D0005E223D1B6F22BD1B80225E189122DE1818
:1006E000AA225E19C322DE19D8225E1AED22DE1A72
:1006F00002230800B601B301B4013C1C822BBC01EB
:10070000BC14842BBC013C143C08B6006400882B4C
:10071000892B8A2B8B2B8C2BFF30B41B8500B41FAD
:100720008501B30B862BB40B862B0310B60CB608D1
:10073000031D862B0030BB003C08BA00E3210800F3
:100740008F08031908008F0178308E00C80FCA2D5A
:10075000C80A441CD02B461CC12BCA1CB22BCA0190
:100760004A15DE2B4A1DB72BCA01CA15DE2BCA1D3E
:10077000BC2BCA014A16DE2B4A1EDE2BCA01CA1444
:10078000DE2B4A1DC62BCA014A16DE2BCA1DCB2BF7
:10079000CA014A16DE2B4A1EDE2BCA01CA14DE2B02
:1007A000CA1CD52BCA014A15DE2B4A1DDA2BCA01F9
:1007B000CA15DE2B4A1EDE2BCA014A15C41C052CA5
:1007C000C61CF62BCB1CE72BCB014B15132C4B1D5A
:1007D000EC2BCB01CB15132CCB1DF12BCB014B16E6
:1007E000132C4B1E132CCB01CB14132C4B1DFB2BAA
:1007F000CB014B16132CCB1D002CCB014B16132C0D
:100800004B1E132CCB01CB14132CCB1C0A2CCB016D
:100810004B15132C4B1D0F2CCB01CB15132C4B1E42
:10082000132CCB014B15441D3A2C461D2B2CCC1CF4
:100830001C2CCC014C15482C4C1D212CCC01CC156A
:10084000482CCC1D262CCC014C16482C4C1E482C78
:10085000CC01CC14482C4C1D302CCC014C16482C0F
:10086000CC1D352CCC014C16482C4C1E482CCC01F0
:10087000CC14482CCC1C3F2CCC014C15482C4C1DC6
:10088000442CCC01CC15482C4C1E482CCC014C15CA
:10089000C41D702CC61D612CCD1C522CCD014D15D4
:1008A0005F137E2C4D1D572CCD01CD157E2CCD1DFB
:1008B0005C2CCD014D167E2C4D1E7E2CCD01CD1411
:1008C0007E2C4D1D662CCD014D167E2CCD1D6B2C26
:1008D000CD014D167E2C4D1E7E2CCD01CD147E2CCF
:1008E000CD1C752CCD014D157E2C4D1D7A2CCD01C6
:1008F000CD157E2C4D1E7E2CCD014D155F1BA72CDA
:10090000441EA72C461E982CCE1C892CCE014E15B9
:10091000B52C4E1D8E2CCE01CE15B52CCE1D932C94
:10092000CE014E16B52C4E1EB52CCE01CE14B52CD4
:100930004E1D9D2CCE014E16B52CCE1DA22CCE01E7
:100940004E16B52C4E1EB52CCE01CE14B52CCE1C99
:10095000AC2CCE014E15B52C4E1DB12CCE01CE15B2
:10096000B52C4E1EB52CCE014E15C41EDC2CC61E59
:10097000CD2CCF1CBE2CCF014F15EA2C4F1DC32C04
:10098000CF01CF15EA2CCF1DC82CCF014F16EA2C72
:100990004F1EEA2CCF01CF14EA2C4F1DD22CCF01D1
:1009A0004F16EA2CCF1DD72CCF014F16EA2C4F1E25
:1009B000EA2CCF01CF14EA2CCF1CE12CCF014F152C
:1009C000EA2C4F1DE62CCF01CF15EA2C4F1EEA2C46
:1009D000CF014F15441F112D461F022DD01CF32CA3
:1009E000D00150151F2D501DF82CD001D0151F2DF2
:1009F000D01DFD2CD00150161F2D501E1F2DD001D3
:100A0000D0141F2D501D072DD00150161F2DD01DA5
:100A10000C2DD00150161F2D501E1F2DD001D014AB
:100A20001F2DD01C162DD00150151F2D501D1B2D14
:100A3000D001D0151F2D501E1F2DD0015015C41FE1
:100A4000462DC61F372DD11C282DD1015115542DEF
:100A5000511D2D2DD101D115542DD11D322DD10176
:100A60005116542D511E542DD101D114542D511D08
:100A70003C2DD1015116542DD11D412DD1015116BE
:100A8000542D511E542DD101D114542DD11C4B2D58
:100A9000D1015115542D511D502DD101D115542D79
:100AA000511E542DD1015115451F7C2D471F6D2D11
:100AB000D21C5E2DD2015215DF138A2D521D632DDB
:100AC000D201D2158A2DD21D682DD20152168A2D3F
:100AD000521E8A2DD201D2148A2D521D722DD2019E
:100AE00052168A2DD21D772DD20152168A2D521EF2
:100AF0008A2DD201D2148A2DD21C812DD2015215F9
:100B00008A2D521D862DD201D2158A2D521E8A2D74
:100B1000D2015215DF1BB32DC51FB32DC71FA42D46
:100B2000D31C952DD3015315C12D531D9A2DD301DF
:100B3000D315C12DD31D9F2DD3015316C12D531E87
:100B4000C12DD301D314C12D531DA92DD30153168B
:100B5000C12DD31DAE2DD3015316C12D531EC12D52
:100B6000D301D314C12DD31CB82DD3015315C12DDE
:100B7000531DBD2DD301D315C12D531EC12DD3013E
:100B80005315D5214008C4004108C5005F18DF1483
:100B90005F1CDF104808C9000C304A05031D051210
:100BA0000C304B05031D85120C304C05031D051040
:100BB0000C304D05031D85100C304E05031D8710AC
:100BC0000C304F05031D07110C305005031D071095
:100BD0000C305105031D87120C305205031D0712FE
:100BE0000C305305031D871149080E020318242EEB
:100BF00012304A05031D051612304B05031D8516DC
:100C000012304C05031D051412304D05031D8514CB
:100C100012304E05031D871412304F05031D0715B2
:100C200012305005031D071412305105031D87169D
:100C300012305205031D071612305305031D871588
:100C4000FF304802031908008F08031D0800962092
:100C500049080E02031C242E18304A05031D0512F4
:100C600006304A05031D051618304B05031D851275
:100C700006304B05031D851618304C05031D051065
:100C800006304C05031D051418304D05031D851055
:100C900006304D05031D851418304E05031D8710C1
:100CA00006304E05031D871418304F05031D07112C
:100CB00006304F05031D071518305005031D07109A
:100CC00006305005031D071418305105031D871207
:100CD00006305105031D871618305205031D0712F3
:100CE00006305205031D071618305305031D8711E2
:0A0CF00006305305031D87150800A8
:084000000900030004000500A3
:02400E00CC33B1
:10420000010078007A007C007E007B0079007F004E
:104210007D007A0078007E007C007D007F00FF003A
:104220000200F200F600FA00FE00F200F600FA00CA
:10423000FE00F200F600FA00FE00F200F600FF00B9
:10424000FF00050005000500050009000900090040
:1042500009000D000D000D000D0011001100FF0000
:104260000100FF00FF00FF00FF00FF00FF00FF0054
:10427000FF00FF00FF00FF00FF00FF00FF00FF0046
:10428000FF00FF00FF00FF00FF00FF00FF00FF0036
:10429000FF00FF00FF00FF00FF00FF00FF00FF0026
:1042A000FF00FF00FF00FF00FF00FF00FF00FF0016
:1042B000FF00FF00FF00FF00FF00FF00FF00FF0006
:1042C000FF00FF00FF00FF00FF00FF00FF00FF00F6
:1042D000FF00FF00FF00FF00FF00FF00FF00FF00E6
:1042E000FF00FF00FF00FF00FF00FF00FF00FF00D6
:1042F000FF00FF00FF00FF00FF00FF00FF00DD00E8
:00000001FF
